:040000000CEF00F011
:10000800D8CFFFF5E0CF0FF0FACFFEF5AFEF07F04E
:1000180000EE11F011EE24F0B0EC28F005EEB2F08D
:1000280015EEE2F0B0EC28F000EEF0F011EE00F082
:10003800640EF66E000EF76E000EF86EA7EC28F050
:1000480005EE93F015EEB2F0740EF66E000EF76E34
:10005800000EF86EA7EC28F066EF04F060082F0891
:1000680013087208AB088A084608F6070000746689
:10007800747077722E62696E007466747072642E82
:0C00880074787400002D5C7C2F010200D5
:10009400FFFF0FD000018E6F3F0EC716C66AC56AF8
:1000A400C686C75094869488C68A8E51C86E12003C
:1000B400FFFFF0D7AF00FFFF92D0AFC0B1F0B0C0E8
:1000C400B2F00001B36F00D0C5CF00F01F0E0016D0
:1000D40000C002F0036A000EC7B4010E0212000E43
:1000E400031203500210D8A401D001D0EDD7C5806B
:1000F40000D0C5B001D001D0FCD7A1A601D001D059
:1001040002D0010E6AD00001B3511CDA0009D8B440
:1001140001D001D002D0010E60D000D0C5CF00F0D4
:100124001F0E001600C002F0036A000EC7B4010ED1
:100134000212000E031203500210D8A401D001D001
:10014400EDD7C5BC01D001D046D00001B251FAD9D7
:100154000009D8B401D001D002D0010E3ED000D0A5
:10016400C5CF00F01F0E001600C002F0036A000E97
:10017400C7B4010E0212000E031203500210D8A4D9
:1001840001D001D0EDD70001B151DCD90009D8B4B8
:1001940001D001D002D0010E20D000D0C5CF00F094
:1001A4001F0E001600C002F0036A000EC7B4010E51
:1001B4000212000E031203500210D8A401D001D081
:1001C400EDD7C5BC01D001D003D0000E06D002D0BB
:1001D400020E03D002D0020E00D01200FFFF6DD732
:1001E4009100FFFF63D00001946F91C0AFF092C003
:1001F400B0F0945160DF0001936F9351D8B401D0F3
:1002040001D002D0935150D011D90001936F935172
:10021400D8B401D001D002D0935146D000D0C5CF7C
:1002240000F01F0E001600C002F0036A000EC7B4EF
:10023400010E0212000E031203500210D8A401D0C2
:1002440001D0EDD7C58000D0C5B001D001D0FCD716
:10025400A1A601D001D002D0010E26D0000194291C
:1002640071D90009D8B401D001D002D0010E1CD03C
:1002740000D0C5CF00F01F0E001600C002F0036AC4
:10028400000EC7B4010E0212000E03120350021036
:10029400D8A401D001D0EDD7C5BC01D001D002D083
:1002A400000E02D0020E00D01200FFFF9CD7FFFF09
:1002B4003ED00001AF6F00D0C5CF00F01F0E001676
:1002C40000C002F0036A000EC7B4010E0212000E51
:1002D400031203500210D8A401D001D0EDD70001BD
:1002E400AF5130D90009D8B401D001D002D0010EE9
:1002F4001CD000D0C5CF00F01F0E001600C002F0C5
:10030400036A000EC7B4010E0212000E031203505A
:100314000210D8A401D001D0EDD7C5BC01D001D0C2
:1003240002D0000E02D0020E00D01200FFFFC1D78F
:10033400FFFF1ED000D0C5CF00F01F0E001600C076
:1003440002F0036A000EC7B4010E0212000E03127B
:1003540003500210D8A401D001D0EDD7C58400D039
:10036400C5B401D001D0FCD7000E00D01200FFFFAD
:10037400E1D7FFFF11D0FCD800D0C5B601D001D021
:10038400FCD7C59AC58800D0C5B801D001D0FCD728
:10039400C95000D01200FFFFEED7FFFF17D0E8D8F6
:1003A40000D0C5B601D001D0FCD7C58AC58800D01D
:1003B400C5B801D001D0FCD7C58400D0C5B401D0E4
:1003C40001D0FCD7000E00D01200FFFFE8D78E004A
:1003D400FFFF2BD000018F6F8EC091F08FC092F081
:1003E4008F51FFDE00018E6F8E51D8B401D001D041
:0C03F40002D08E5118D00BD0BCDF90C09E
:10040000E9FF91C0EAFFEF6E010E00019027000E98
:100410009123000192079229D8A401D001D0EED7F0
:10042000BEDF00018E6F8E5100D01200FFFFD4D7C7
:10043000FFFF24D000D0C5CF00F01F0E001600C073
:1004400002F0036A000EC7B4010E0212000E03127E
:1004500003500210D8A401D001D0EDD7C58400D03C
:10046000C5B401D001D0FCD7A1A601D001D002D0E3
:10047000010E02D0000E00D01200FFFFDBD7FFFFFD
:1004800062D000018F6F00D0C5CF00F01F0E0016A4
:1004900000C002F0036A000EC7B4010E0212000E83
:1004A000031203500210D8A401D001D0EDD7C580AB
:1004B00000D0C5B001D001D0FCD7A1A601D001D099
:1004C00003D0010E3ED02ED000018F513DD800093F
:1004D000D8B401D001D002D0010E33D000D0C5CFA6
:1004E00000F01F0E001600C002F0036A000EC7B431
:1004F000010E0212000E031203500210D8A401D004
:1005000001D0EDD7A1A601D001D002D0010E19D0A3
:10051000C5BC01D001D003D000018E6B03D0040E06
:1005200000018E6FC58400D0C5B401D001D0FCD7C6
:10053000A1A601D001D002D0010E03D000018E513E
:1005400000D01200FFFF9DD7FFFF13D0C96E00013E
:10055000B46FC6AE01D001D003D0FF0E08D007D0D3
:1005600000D0C7B001D001D0FCD7000E00D01200DF
:10057000FFFFECD7FFFF0AD0C58600D0C7A001D08F
:1005800001D0FCD7C95000D01200FFFFF5D7C6003C
:10059000FFFFC8C0F3FFC9C0F4FFC6C0D9FFC7C082
:1005A000DAFF0001CA51006ECB51016ECA07000E7E
:1005B000CB5B01500010D8B41AD0F3CFF6FFF4CFC4
:1005C000F7FFF32A000EF422D9CFE9FFDACFEAFFD2
:1005D000D94ADA2A050EF76403D00800F55005D091
:1005E000F6CFE1FFF7CFE2FFE750EF6EDAD7C6C0F4
:0C05F00000F0C7C001F01200FFFFCBD7E5
:100600004D434850537461636B2076322E32320072
:10061000444843502F476C65616E696E672E2E2EDD
:1006200000426F6172642053657475702E2E2E0027
:1006300020202020202020202020202020202020BA
:100640000050555400474554000D0A0D0A0D4D4306
:100650004850537461636B205446545020436C6976
:10066000656E742044656D6F2076312E3020284DE4
:10067000434850537461636B2076322E32322C2003
:100680004175672031322032303033290D0A0D0A8E
:1006900009313A204368616E676520426F61726478
:1006A0002073657269616C206E756D6265722E0DC6
:1006B0000A09323A204368616E67652064656661A5
:1006C000756C7420495020616464726573732E0DDB
:1006D0000A09333A204368616E6765206465666184
:1006E000756C7420676174657761792061646472E8
:1006F0006573732E0D0A09343A204368616E67658D
:100700002064656661756C74207375626E65742013
:100710006D61736B2E0D0A09353A20456E61626C6E
:10072000652044484350202620495020476C65618D
:100730006E696E672E0D0A09363A2044697361624C
:100740006C652044484350202620495020476C6562
:10075000616E696E672E0D0A09373A205365742061
:10076000544654502053657276657220495020617A
:100770006464726573733A0D0A09383A20536176DE
:1007800065202620517569742E0D0A0D0A456E7478
:1007900065722061206D656E752063686F696365A1
:1007A0002028312D38293A20000D0A496E76616CD7
:1007B000696420696E707574207265636569766519
:1007C00064202D20496E7075742069676E6F7265A4
:1007D000642E0D0A507265737320616E79206B650B
:1007E0007920746F20636F6E74696E75652E2E2E7E
:1007F0000D0A002575000D0A4E6F772072756E6E1A
:10080000696E67206170706C69636174696F6E2EC8
:100810002E2E000D0A44656661756C742047617464
:100820006577617920416464726573732028000DD7
:100830000A44656661756C74204950204164647295
:100840006573732028000D0A544654502053657276
:1008500065722049502041646472657373202800DA
:100860000D0A53657269616C204E756D6265722068
:1008700028000D0A44656661756C74205375626EBC
:100880006574204D61736B2028000D0A4448435065
:10089000202620495020476C65616E696E67206490
:1008A000697361626C65642E0D0A000D0A44484349
:1008B00050202620495020476C65616E696E672084
:0C08C000656E61626C65642E0D0A00001C
:1008CC00FFFF99D00501E181DBEC08F00B0E4AEC3F
:1008DC0000F057EC28F0FDEC08F081BA01D001D003
:1008EC000CD0C00ED9EC25F00001210EB96F060E0C
:1008FC00BA6F4BEC26F057EC0BF034EC23F05DC0E8
:10090C0000F000A001D001D00BD0C00ED9EC25F026
:10091C000001100EB96F060EBA6F4BEC26F006D024
:10092C00010EE8CFE0F5070EE8CF93F561D064EC4B
:10093C0028F03DC0E8FF005C046E3EC0E8FF0158A3
:10094C00056E3FC0E8FF0258066E40C0E8FF035832
:10095C00076E000E075C08E1000E065C05E1000E58
:10096C00055C02E1320E045CD8A001D001D00BD0A2
:10097C0064EC28F000C03DF001C03EF002C03FF036
:10098C0003C040F0897843EC23F0B3C5E8FF0501C0
:10099C00E019D8B401D001D024D00001450EAC6FC1
:1009AC00000EAD6F010EAE6F0FDBB3C5E0F55DC091
:1009BC0000F000A001D001D014D0CE0ED9EC25F05F
:1009CC000A0E0501E06101D001D006D0E0C5E8FFB8
:1009DC00300F70EC26F005D0E0C5E8FF410F70EC4D
:1009EC0026F0B9C500F000B001D001D001D004D878
:1009FC009ED70CEF00F066D7FFFFDCD0ABC5E8FF4D
:100A0C00030AD8A401D006D0ABC5E8FF040AD8A4C9
:100A1C0002D000D002D000D042D064EC28F041C00B
:100A2C00E8FF005C046E42C0E8FF0158056E43C04D
:100A3C00E8FF0258066E44C0E8FF0358076E000E2C
:100A4C00075C08E1000E065C05E1000E055C02E1A6
:100A5C00320E045CD8A001D001D021D08F0ED9EC7D
:100A6C0025F00501DF2BDF0505EEACF0E926000EC5
:100A7C00EA22EF5070EC26F0DFC5E8FF040AD8A498
:100A8C0001D001D002D00501DF6B64EC28F000C06E
:100A9C0041F001C042F002C043F003C044F079D0F1
:100AAC0000015E0E8F6F000E906F22EC14F0010EA1
:100ABC00E8CFABF57DD04BEC14F000018E6F8E516E
:100ACC00D8A401D001D004D0020EE8CFABF509D0E8
:100ADC0000018E51050AD8A401D001D002D0050125
:100AEC00AB6B66D081BA01D001D028D0800ED9EC86
:100AFC0025F00001300EB96F060EBA6F4BEC26F0E4
:100B0C00800ED9EC25F0E1C500F000A001D001D099
:100B1C000BD00001410EB96F060EBA6F4BEC26F0EC
:100B2C00030EE8CFABF50AD00001450EB96F060EE7
:100B3C00BA6F4BEC26F0040EE8CFABF539D03BD8AE
:100B4C000009D8B401D001D003D0050EE8CFABF525
:100B5C002FD028D90009D8B401D001D003D0050E6C
:100B6C00E8CFABF525D081AA01D001D010D0E1C5DA
:100B7C0000F0000E00A0010E006E05EEE1F0EF504B
:100B8C000018FE0B0018EF6E020EE8CFABF510D07C
:100B9C000FD0ABC5E8FF000A83E0010A8CE0030A22
:100BAC00A1E0010ACCE0070AD4E0010ADCE000D0A5
:100BBC001200FFFF23D7FFFFF4D00001906B010E52
:100BCC00926F9FD0DCC5DEF5CEEC10F00009D8B4E6
:100BDC0001D001D011D000013B6B3C6B396B3A6BEF
:100BEC000001950E936F050E946F020E956FBFEC7E
:040BFC0014F0020EE1
:100C0000E8CFB0F591D0FDEC14F00001916F915157
:100C1000D8A401D001D004D0030EE8CFB0F50AD09B
:100C200000019151040AD8A401D001D003D0010ED3
:100C3000E8CFB0F579D04DD0BCEC16F00001916F43
:100C40009151D8A401D001D036D09251D8B401D05E
:100C500001D005D0926B3BC039F03CC03AF03BC0AC
:100C6000F6FF3CC0F7FF050EF76404D00800FFFF55
:100C7000F55005D0F6CFE9FFF7CFEAFFEF500001BE
:100C80008F6F0001010E3B27000E3C233F0E3C5DA1
:100C9000FF0ED8B43B5DD8A001D001D007D06BECDB
:100CA00016F0040EE8CFB0F515D004D000018F5136
:100CB000AAEC17F00ED000019151040AD8A401D07B
:100CC00001D006D039C03BF03AC03CF003D001D08F
:100CD00001D0B2D729D0ACEC16F00001916F915140
:100CE000D8A401D001D003D0010E906F0ED0000126
:100CF0009151040AD8A401D001D007D039C03BF0EB
:100D00003AC03CF0030EE8CFB0F50ED00DD0B0C520
:100D1000E8FF010A01E15CD7030A01E174D7010A87
:100D20008AE0070AD8E000D000019151D8A406D08B
:100D300000D09051D8B402D000D002D000D007D05B
:100D40008F0ED9EC25F0590E70EC26F022D0000160
:100D50009151050AD8A401D005D09151030AD8A415
:100D600002D000D002D000D014D08F0ED9EC25F0E4
:100D700000019151050AD8A401D001D004D0540E2D
:100D800070EC26F003D0450E70EC26F0010E000149
:100D9000906F00019051D8B401D001D003D0010E62
:100DA000E8CFB0F50001905100D01200FFFF0BD743
:100DB000FFFF8FD00001906B43D0DCC5DEF5CEEC99
:100DC00010F00009D8B401D001D00CD00001A00E61
:100DD000936F050E946F010E956FBFEC14F0030E28
:100DE000E8CFB1F536D0FDEC14F00001916F9151D0
:100DF000D8A401D001D004D0040EE8CFB1F50DD0B5
:100E000000019151040AD8A401D001D005D0020EEE
:100E1000E8CFB1F51ED001D01CD00FD00DEC15F0ED
:100E20000001916F9151D8A401D001D005D046ECBA
:100E300016F000018F6F01D001D0F0D70AD009D091
:100E4000B1C5E8FF020AB9E0010ACDE0070AE5E012
:100E500000D000019151020AD8A401D001D009D0DC
:100E6000010E906F8F0ED9EC25F0590E70EC26F024
:100E700022D000019151050AD8A401D005D091518A
:100E8000030AD8A402D000D002D000D014D0010EA2
:100E90000001906F8F0ED9EC25F000019151050AE9
:100EA000D8A401D001D004D0540E70EC26F003D0A9
:100EB000450E70EC26F000019051D8B401D001D05D
:100EC00003D0020EE8CFB1F50001905100D012001E
:100ED000FFFF70D7FFFF42D072EC28F0E2C5F3FFAE
:100EE000E3C5F4FFE4C5F5FFE5C5F6FFE6C5F7FF8A
:100EF000E7C5F8FFE8C500F0E9C501F0EAC502F072
:100F0000EBC503F0ECC504F0EDC505F0EEC506F049
:100F1000EFC507F0F0C508F0F1C509F0F2C50AF019
:100F2000F3C50BF0F4C50CF0F5C50DF0F6C50EF0E9
:100F3000F7C5DAFFF8C5D9FFF9C5E2FFFAC5E1FF49
:100F4000FBC5EAFFFCC5E9FFFDC5E8FFFACFFEF5EA
:100F50000FC0E0FFFFC5D8FF1000FFFFBDD7FFFFA8
:100F6000E8CFFDF5E9CFFCF5EACFFBF5E1CFFAF5E7
:100F7000E2CFF9F5D9CFF8F5DACFF7F50EC0F6F5EF
:100F80000DC0F5F50CC0F4F50BC0F3F50AC0F2F591
:100F900009C0F1F508C0F0F507C0EFF506C0EEF5A1
:100FA00005C0EDF504C0ECF503C0EBF502C0EAF5B1
:100FB00001C0E9F500C0E8F5F8CFE7F5F7CFE6F5B1
:100FC000F6CFE5F5F5CFE4F5F4CFE3F5F3CFE2F5B1
:100FD00081D7AC00FFFFEED00001AE51D8B401D0F4
:100FE00001D00AD0C00ED9EC25F00001300EB96F47
:100FF000060EBA6F4BEC26F0C00ED9EC25F00001BE
:10100000AF0EBB6F000EBC6FF30EBD6F070EBE6F51
:10101000ACC0E9FFADC0EAFFEF50006E00C002F0C7
:10102000036A02C0B7F003C0B8F0B70EE8CFB9F05A
:10103000000EE8CFBAF08EEC1BF00001AE51D8B430
:1010400001D001D00AD0AF0EB96F000EBA6F30ECEC
:1010500026F02E0E70EC26F008D00001AF0EB96F0E
:10106000000EBA6F51DB2E0E3FDB0001AF0EBB6FDF
:10107000000EBC6FF30EBD6F070EBE6F00EE01F0E9
:10108000AC51E926AD51EA22EF50006E00C002F0EB
:10109000036A02C0B7F003C0B8F0B70EE8CFB9F0EA
:1010A000000EE8CFBAF08EEC1BF00001AE51D8B4C0
:1010B00001D001D00AD0AF0EB96F000EBA6F30EC7C
:1010C00026F02E0E70EC26F008D00001AF0EB96F9E
:1010D000000EBA6F19DB2E0E07DB0001AF0EBB6FDF
:1010E000000EBC6FF30EBD6F070EBE6F00EE02F078
:1010F000AC51E926AD51EA22EF50006E00C002F07B
:10110000036A02C0B7F003C0B8F0B70EE8CFB9F079
:10111000000EE8CFBAF08EEC1BF00001AE51D8B44F
:1011200001D001D00AD0AF0EB96F000EBA6F30EC0B
:1011300026F02E0E70EC26F008D00001AF0EB96F2D
:10114000000EBA6FE1DA2E0ECFDA0001AF0EBB6FE0
:10115000000EBC6FF30EBD6F070EBE6F00EE03F006
:10116000AC51E926AD51EA22EF50006E00C002F00A
:10117000036A02C0B7F003C0B8F0B70EE8CFB9F009
:10118000000EE8CFBAF08EEC1BF00001AE51D8B4DF
:1011900001D001D007D0AF0EB96F000EBA6F30EC9E
:1011A00026F006D00001AF0EB96F000EBA6FACDAB0
:1011B0001200FFFF11D7FFFF1FD08E0EC16E030E6E
:1011C000926E809A89848986F19E9CEC25F0800E2F
:1011D000D9EC25F00001000EB96F060EBA6F4BEC8A
:1011E00026F0200EAC6E900EAB6E0F0EAF6ED56A71
:1011F000F28EF28C1200FFFFE0D7FFFF6CD00A0ED8
:10120000E8CF45F00A0EE8CF46F0050EE8CF47F0EC
:101210000F0EE8CF48F0FF0EE8CF4FF0FF0EE8CFFB
:1012200050F0FF0EE8CF51F00001526B0A0EE8CFEC
:1012300053F00A0EE8CF54F0050EE8CF55F00F0E2C
:10124000E8CF56F0496B040EE8CF4AF0A30EE8CF82
:101250004BF04C6B4D6B4E6B5D810001450E8F6FFB
:10126000000E906F916B926BA00EF3EC00F0BBEC54
:1012700001F000018E6FCFEC01F000018E51550A94
:10128000D8A401D001D024D0010E916F926BA00E92
:10129000F3EC00F000018E6B1C0E8E6501D001D0C6
:1012A00001D013D0BBEC01F08FC0E9FF90C0EAFF82
:1012B000EF6E010E00018F27000E9023010E8E2786
:1012C0001C0E8E6501D001D0EDD7CFEC01F001D01E
:1012D00003D81200FFFF93D7FFFF2BD00001450E6C
:1012E000AD6F000EAE6FAF6BB06BA00E5DEC00F09B
:1012F000550E59EC01F00001AC6B1C0EAC6501D031
:1013000001D001D012D0ADC0E9FFAEC0EAFF0001AC
:10131000AD4BAE2BEF5059EC01F0010E0001AC27A4
:101320001C0EAC6501D001D0EED79AEC01F0120092
:10133000FFFFD4D7AC00FFFF21D003D00001AE5196
:10134000D3D90001ACC0F6FFADC0F7FF010EAC274A
:10135000000EAD23050EF76404D00800FFFFF55022
:1013600005D0F6CFE9FFF7CFEAFFEF50AE6FAE51F1
:10137000D8A401D001D0E2D71200FFFFDED7AC0025
:10138000FFFF38D00001B06B00D09EAA01D001D081
:10139000FCD7AE500001AF6FAF510D0AD8A401D0F9
:1013A00005D0AF510A0AD8A402D000D002D000D094
:1013B00001D01BD0010E0001B027ACC0E9FFADC0C9
:1013C000EAFFAFC0EFFF010EAC27000EAD23ACC0AB
:1013D000E9FFADC0EAFF000EEF6EAE07AE29D8A45C
:1013E00001D001D001D001D0CFD70001B05100D041
:1013F0001200FFFFC7D7AC00FFFF64D0ACC0B1F054
:10140000ADC0B2F00001B36B3AD00001B0512E0A6A
:10141000D8A401D001D020D0ACC0E9FFADC0EAFF14
:10142000000EEF6E010EAC27000EAD23B1C0B4F07C
:10143000B2C0B5F079EC27F00001B351AE25E96EEA
:10144000000EAF21EA6E00C0EFFF010EB327ACC063
:10145000B1F0ADC0B2F00ED0300E0001B06101D0DD
:1014600004D0390EB06502D000D002D000D002D036
:10147000000E26D0010E0001AC27000EAD23ACC03B
:10148000E9FFADC0EAFFEF500001B06FB051D8A442
:1014900001D001D0BAD7B1C0B4F0B2C0B5F079EC88
:1014A00027F00001B351AE25E96E000EAF21EA6EC0
:1014B00000C0EFFFB351030A000ED8B4010E00D0F4
:1014C0001200FFFF9BD7FFFF1BD000D09EAA01D0C8
:1014D00001D0FCD7AE5000018F6F300E8F6506D063
:1014E00000D0390E8F6102D000D002D000D004D0DD
:1014F00000018F5103D002D0390E00D01200FFFF3F
:10150000E4D7FFFFD3D00001A96F0D0EEDD80A0E6E
:10151000EBD80001A951020D8E0EF324E96E000EE6
:10152000F420EA6EEECFACF0EDCFADF004DFA8D042
:1015300000018F0EBB6F000EBC6FF30EBD6F070E68
:10154000BE6F00EE57F0EECFAAF0EDCFABF0AA0ED3
:10155000E8CFB9F0000EE8CFBAF08EEC1BF0000136
:101560008F0EB96F000EBA6FCFD8290EBDD83A0EC4
:10157000BBD8200EB9D800018F0EAC6F000EAD6F36
:10158000140EAE6FFDDE006E00C002F0036A035061
:101590000210D8B401D001D00FD08F0EB46F000E5E
:1015A000B56F79EC27F000C057F001C058F058C073
:1015B0004DF057C04EF001D03AD076D00001450E24
:1015C000A76F000EA86F0BD00001530EA76F000E7F
:1015D000A86F05D000014F0EA76F000EA86FA7C01F
:1015E000ACF0A8C0ADF00001AE6BF4DC290E7CD8E5
:1015F0003A0E7AD8200E78D800018F0EAC6F000E0C
:10160000AD6F140EAE6FBCDE8F0EAC6F000EAD6F03
:10161000A30EAE6F000EAF6FEFDE006E00C002F0E3
:10162000036A03500210D8A401D001D00DD00001EC
:10163000A90EAC6F070EAD6F7EDE00D09EAA01D062
:1016400001D0FCD7AE500CD0A7C0E9FFA8C0EAFF7C
:10165000A3C0EEFFA4C0EEFFA5C0EEFFA6C0EEFF44
:1016600023D000015D8120D000015D911DD00001DB
:101670005E0EA76F000EA86FB2D72EDE15D014D065
:101680000001A951310A01E153D7030A97E0010A89
:101690009BE0070A9FE0010AE4E0030AE5E0010A93
:1016A000E6E00F0AEAE000D01200FFFF2CD7FFFFB0
:1016B0001AD00001490EAC6F060EAD6F3CDE03DFA1
:1016C00000018E6F8E51390AD8B401D001D002D0FA
:1016D0008E5117DF00018E51380AD8A401D001D0F5
:1016E000E8D71200FFFFE5D7FFFF0CD00001BC6F69
:1016F00000D0ACA201D001D0FCD70001BC51AD6E2E
:101700001200FFFFF3D7B900FFFF14D003D0000190
:10171000BB51EADFB9C0E9FFBAC0EAFF0001B94B2B
:10172000BA2BEF50BB6FBB51D8A401D001D0EFD77B
:101730001200FFFFEBD7FFFF05D00F0ED8EC1FF014
:101740001200FFFFFAD7FFFF05D0040ED8EC1FF000
:101750001200FFFFFAD7FFFF11D0F29E04D0D00E87
:101760000001BD6F03D0010E0001BD6F01D000D09C
:101770000001BD2FFCD7F28E1200FFFFEED7FFFF56
:1017800093D179D1000194699569966997699869AF
:1017900099699A699B699C699D690001316B326BFB
:1017A000336B346B440E00019F6FA06B940EA16FDE
:1017B000000EA26F430EA36FA46B46EC18F0E8CFA7
:1017C000B4F564EC28F000C021F001C022F002C0A2
:1017D00023F003C024F0010EE8CF93F564EC28F069
:1017E00021C0E8FF005C046E22C0E8FF0158056ECE
:1017F00023C0E8FF0258066E24C0E8FF0358076EB6
:10180000000E075C08E1000E065C05E1000E055CB9
:1018100002E1140E045CD8A001D001D003D0020E66
:10182000E8CF93F53FD1000131513211331134111A
:10183000D8B401D001D004D0040EE8CF93F518D06D
:10184000B4C5DEF5CEEC10F00009D8B401D001D05B
:101850000FD0010EF8DA64EC28F000C021F001C0CE
:1018600022F002C023F003C024F0030EE8CF93F56A
:1018700019D1B4C5E8FFCBEC19F00009D8B401D0F8
:1018800001D00AD01ED9020AD8A401D001D003D0B9
:10189000040EE8CF93F524D064EC28F021C0E8FFD3
:1018A000005C046E22C0E8FF0158056E23C0E8FF0B
:1018B0000258066E24C0E8FF0358076E000E075C4E
:1018C00008E1000E065C05E1000E055C02E1C80EB1
:1018D000045CD8A001D001D003D0020EE8CF93F56C
:1018E000E1D0B4C5DEF5CEEC10F00009D8B401D0DB
:1018F00001D00FD0030EA7DA64EC28F000C021F06D
:1019000001C022F002C023F003C024F0050EE8CF8E
:1019100093F5C8D0B4C5E8FFCBEC19F00009D8B4F2
:1019200001D001D044D0CDD800019E6F9E51060A4F
:10193000D8A401D001D004D0040EE8CF93F536D05E
:1019400000019E51050AD8A401D001D02FD0B4C502
:10195000E8FFB2EC18F064EC28F000C021F001C000
:1019600022F002C023F003C024F0060EE8CF93F566
:1019700031C045F032C046F033C047F034C048F0C3
:1019800035C04FF036C050F037C051F038C052F07B
:101990002DC053F02EC054F02FC055F030C056F07B
:1019A000050194810501010EB3277CD024D064EC9D
:1019B00028F021C0E8FF005C046E22C0E8FF015857
:1019C000056E23C0E8FF0258066E24C0E8FF0358E6
:1019D000076E000E075C08E1000E065C05E1000ED4
:1019E000055C02E1C80E045CD8A001D001D003D090
:1019F000020EE8CF93F556D064EC28F021C0E8FF42
:101A0000005C046E22C0E8FF0158056E23C0E8FFA9
:101A10000258066E24C0E8FF0358076E000E075CEC
:101A200008E1000E065C05E1000E055C02E1640EB3
:101A3000045CD8A001D001D01DD00001FF0E2527E5
:101A4000FF0E2623FF0E2723FF0E282325512611E4
:101A500027112811D8A401D001D002D00501936B21
:101A600064EC28F000C021F001C022F002C023F095
:101A700003C024F017D093C5E8FF000A01E182D625
:101A8000010A01E1ABD6030A01E1CDD6010A01E169
:101A9000F0D6070A01E125D7010A01E13BD7030A85
:101AA000ABE000D01200FFFF6CD6FFFF09D0080E9C
:101AB000E8CF93F5B4C5E8FFB2EC18F01200FFFFD1
:101AC000F6D7FFFFBFD10001A16B0001000E286F08
:101AD000000E276F000E266F3C0E256F00019F0E33
:101AE000A76F000EA86FE4EC19F000019F51020AE5
:101AF000D8A401D001D078D1A06B0E0EA06501D082
:101B000001D001D00FD000019F0EA76F000EA86F6B
:101B1000E4EC19F0010E0001A0270E0EA06501D023
:101B200001D0F1D70001310EA76F000EA86FE4ECD1
:101B300019F00001320EA76F000EA86FE4EC19F047
:101B40000001330EA76F000EA86FE4EC19F000013E
:101B5000340EA76F000EA86FE4EC19F00001A06B23
:101B6000DB0EA06501D001D001D00FD000019F0E87
:101B7000A76F000EA86FE4EC19F0010E0001A0277A
:101B8000DB0EA06501D001D0F1D70001A26B0001EE
:101B90009F0EA76F000EA86FE4EC19F00CD10001A6
:101BA0009F0EA76F000EA86FE4EC19F000019F05CF
:101BB000D8A401D001D007D0A10EA76F000EA86F46
:101BC000E4EC19F001D038D109D100019F0EA76FC4
:101BD000000EA86FE4EC19F000019F51040AD8A48C
:101BE00001D001D01CD0350EA76F000EA86FE4EC19
:101BF00019F00001360EA76F000EA86FE4EC19F083
:101C00000001370EA76F000EA86FE4EC19F0000179
:101C1000380EA76F000EA86FE4EC19F001D00CD1BC
:101C2000DDD000019F0EA76F000EA86FE4EC19F045
:101C3000030E00019F6501D001D01CD02D0EA76FAF
:101C4000000EA86FE4EC19F000012E0EA76F000E35
:101C5000A86FE4EC19F000012F0EA76F000EA86F1B
:101C6000E4EC19F00001300EA76F000EA86FE4EC51
:101C700019F001D0E1D0FC0E00019F2707D0000130
:101C8000A00EA76F000EA86FE4EC19F000019F07EB
:101C90009F29D8A401D001D0F2D7A0D000019F0E77
:101CA000A76F000EA86FE4EC19F000019F51040A21
:101CB000D8A401D001D01CD0A60EA76F000EA86F2B
:101CC000E4EC19F00001A50EA76F000EA86FE4EC7C
:101CD00019F00001A40EA76F000EA86FE4EC19F034
:101CE0000001A30EA76F000EA86FE4EC19F001D05D
:101CF000A3D074D0010E0001A26F70D000019F0E1E
:101D0000A76F000EA86FE4EC19F000019F51040AC0
:101D1000D8A401D001D036D0280EA76F000EA86F2E
:101D2000E4EC19F00001270EA76F000EA86FE4EC99
:101D300019F00001260EA76F000EA86FE4EC19F051
:101D40000001250EA76F000EA86FE4EC19F000EE5D
:101D500028F0000EED5C08E1000EED5C05E1070ED9
:101D6000ED5C02E1090EEF5CD8A001D001D009D0F2
:101D70000001F80E2527F80E2623FF0E2723FF0E5D
:101D8000282301D059D02AD000019F0EA76F000E42
:101D9000A86FE4EC19F007D00001A00EA76F000EA9
:101DA000A86FE4EC19F000019F079F29D8A401D087
:101DB00001D0F2D713D000019F51010A01E105D7EC
:101DC000020A01E12ED7300A99E0060A01E1E7D6BE
:101DD000030A01E163D7C90A8DE0D6D70001A251F9
:101DE000D8B401D001D0D3D60001A151020AD8A4A1
:101DF00001D001D009D0A3C029F0A4C02AF0A5C009
:101E00002BF0A6C02CF013D000EE29F00001EE500C
:101E1000A31908E1EE50A41905E1EE50A51902E15D
:101E2000EE50A619D8B401D001D001D0A16B40EC7E
:101E30001AF00001A15104D040EC1AF0000E00D0BD
:101E40001200FFFF40D6FFFFDCD00001A06F010EA3
:101E5000C5EC18F0010EC5EC18F0060EC5EC18F034
:101E6000000EC5EC18F0120EC5EC18F0230EC5ECF0
:101E700018F0340EC5EC18F0560EC5EC18F0000E34
:101E8000C5EC18F0000EC5EC18F0800EC5EC18F08B
:101E9000000EC5EC18F0000EC5EC18F0000EC5ECF5
:101EA00018F0000EC5EC18F0000EC5EC18F000019B
:101EB0009F6B0B0E9F6501D001D001D00BD0000E9F
:101EC000C5EC18F0010E00019F270B0E9F6501D095
:101ED00001D0F5D749C0E8FFC5EC18F04AC0E8FFCB
:101EE000C5EC18F04BC0E8FFC5EC18F04CC0E8FF9B
:101EF000C5EC18F04DC0E8FFC5EC18F04EC0E8FF87
:101F0000C5EC18F000019F6BC90E9F6501D001D090
:101F100001D00BD0000EC5EC18F0010E00019F2778
:101F2000C90E9F6501D001D0F5D7630EC5EC18F03E
:101F3000820EC5EC18F0530EC5EC18F0630EC5EC1C
:101F400018F0350EC5EC18F0010EC5EC18F00001C4
:101F5000A051C5EC18F00001A005D8B40AD000D0FB
:101F600000013151321133113411D8B402D000D0F4
:101F700002D000D016D0360EC5EC18F0040EC5EC19
:101F800018F02CC0E8FFC5EC18F02BC0E8FFC5EC3A
:101F900018F02AC0E8FFC5EC18F029C0E8FFC5EC2E
:101FA00018F0370EC5EC18F0020EC5EC18F0010E53
:101FB000C5EC18F0030EC5EC18F00001A051030A9F
:101FC000D8A401D001D016D0320EC5EC18F0040E02
:101FD000C5EC18F031C0E8FFC5EC18F032C0E8FFDE
:101FE000C5EC18F033C0E8FFC5EC18F034C0E8FFCA
:101FF000C5EC18F0FF0EC5EC18F046EC19F0120015
:10200000FFFF23D7FFFFC9D000018E6B000E8E6546
:1020100001D001D001D022D000018E51020D200E3E
:10202000F324E96E010EF420EA6E8EC000F0D89021
:102030000036D8900034400FEF6E8E51020D210E05
:10204000F324E96E010EF420EA6E010EEF6E010E2C
:102050008E27000E8E6501D001D0DED70501B66B4C
:102060003CDB020ED8EC1FF01F0E64DB0001ED6FAD
:102070001F0E50DB020ED8EC1FF0070E5BDB006E6C
:1020800000AE01D001D087D0210E0001ED6F000E0F
:1020900041DB020ED8EC1FF0480E0001ED6F0E0E72
:1020A00039DB0001ED6B0A0E35DB0001ED6B0B0E29
:1020B00031DB040E0001ED6F0C0E2CDB020E000173
:1020C000ED6F0D0E27DBB6C5E8FF020D200EF324E1
:1020D000E96E010EF420EA6EEF500001ED6F040E80
:1020E00019DB440E0001ED6F010E14DB5F0E0001E1
:1020F000ED6F020E0FDB5E0E0001ED6F030E0ADBCB
:102100000001ED69070E06DB0001ED6B0F0E02DB2F
:10211000610E0001ED6F000EFDDA49C0EDF0010E19
:10212000F9DA4AC0EDF0020EF5DA4BC0EDF0030E1D
:10213000F1DA4CC0EDF0040EEDDA4DC0EDF0050E15
:10214000E9DA4EC0EDF0060EE5DA00018E6B070EFF
:102150008E6501D001D001D00DD00001ED698E5106
:10216000080FD8DA010E00018E27070E8E6501D008
:1021700001D0F3D7440E0001ED6F070ECBDA440E09
:10218000E8CFB7F5220E0001ED6F000EC3DA0001B3
:10219000ED6B0D0EBFDA1200FFFF36D7FFFF09D03F
:1021A000000EC8DA006E000E00A4010E00D012006E
:1021B000FFFFF6D7FFFF16D00001ED6BED2BE76FA9
:1021C0000A0EA8DA0001ED6B0B0EA4DA120E000164
:1021D000ED6F000E9FDA0001E751ED6F100E9ADAF5
:1021E0001200FFFFE9D7E700FFFF59D0010EE9C059
:1021F00000F0EAC001F00016000E01160001E951DE
:102200000024EB6FEA510120EC6F400EED6F070EDA
:1022100081DA0001EB51ED6F0A0E7CDA0001EC511E
:10222000ED6F0B0E77DA120E0001ED6F000E72DA11
:102230000DD0E7C0E9FFE8C0EAFFEF500001ED6F05
:10224000010EE727000EE823100E64DA0001E951C1
:10225000006EEA51016E010EE95F000EEA5B01506B
:102260000010D8A401D001D0E4D7FF0E0001E96F1F
:10227000EA6B04D00001E907D8A0EA070001EA519F
:10228000E911D8A401D006D0070E54DA006E00ACD4
:1022900002D000D002D000D0EDD71200FFFFA6D7A9
:1022A000FFFF13D0010E0001ED6F0A0E33DA0001BB
:1022B000ED6B0B0E2FDA0A0E0001ED6F000E2ADA1D
:1022C000100E38DA00D01200FFFFECD7CE00FFFF6F
:1022D0003BD0D0C0D2F0D1C0D3F0400E0001ED6FA2
:1022E000070E18DA0001D251ED6F0A0E13DA000161
:1022F000D351ED6F0B0E0EDA0A0E0001ED6F000EDA
:1023000009DA0CD0100E16DACEC0E9FFCFC0EAFF12
:10231000EF6E010E0001CE27000ECF230001D05139
:10232000006ED151016E010ED05F000ED15B0150E5
:102330000010D8A401D001D0E5D7D2C000F0D3C09E
:1023400001F000D01200FFFFC4D7FFFF0ED0000144
:102350008E6F8E51020D210EF324E96E010EF420D2
:10236000EA6E000EEF6E1200FFFFF1D7FFFF10D0F4
:1023700000018E6F8E51020D210EF324E96E010EC5
:10238000F420EA6E010EEF6E8EC0B6F51200FFFF6C
:10239000EFD7FFFF18D00501B7050001CD6F440E40
:1023A000CD6101D001D002D05E0ECD6F200E0001B4
:1023B000ED6F000EAFD90001CD51ED6F030EAAD91C
:1023C00000D01200FFFFE7D7FFFF2FD0600E000103
:1023D000ED6F000E9FD9070EADD900018E6F200E54
:1023E000ED6F000E97D9B5C5E8FF00018E6101D0F1
:1023F00001D008D0B5C5E8FF5F08006E8E510024FB
:102400008F6F05D0B5C5E8FF00018E5D8F6F0001AD
:102410008F511B088F6F8F51916F906B90C000F0A0
:1024200091C001F000D01200FFFFD0D79400FFFF51
:10243000B3D096C0E9FF97C0EAFFFF0EEF6E070E1C
:1024400079D9006E00A801D001D024D0210E00015E
:10245000ED6F000E5FD9FF0E97D90001ED6B0A0EEC
:1024600059D90001ED6B0B0E55D9020E0001ED6F2D
:102470000D0E50D9200E0001ED6F000E4BD989DFF3
:102480000001ED69070E46D90001ED6B0D0E42D932
:10249000000E80D0600E0001ED6F000E3BD9070EDC
:1024A00049D90001AA6F200EED6F000E33D900014B
:1024B000AA510501B719D8B401D001D069D0B7C568
:1024C000ACF00001AB6BABC0E7F0ACC0E8F044D9B6
:1024D0000001980ECE6F000ECF6F120ED06FD16B31
:1024E000F6DE000198A10DD000D000EE9AF0EE5279
:1024F000000EED5C400ED8B4EF5CD8A002D000D046
:1025000001D00CD000EE9AF0EE52050EED5CEF0E0D
:10251000D8B4EF5CD8B002D000D002D000D032D016
:10252000A8C0E1F0A9C0E2F088EC1EF000C0A8F05D
:1025300001C0A9F094C0C6F095C0C7F00001A20E7A
:10254000C86F000EC96F060ECA6FCB6BC8EC02F0E5
:102550000001A951080AD8A40DD000D0A851D8A4D0
:1025600001D005D0A851060AD8A402D000D001D0CD
:1025700001D002D000D006D096C0E9FF97C0EAFF94
:10258000A8C0EFFFB7C5B5F599C0B7F5010E02D0E9
:10259000000E00D01200FFFF4CD7DF00FFFF63D01A
:1025A0000A0E0001ED6F070EB5D8B6C5E8FF020DA3
:1025B000200EF324E96E010EF420EA6EEF500001C4
:1025C000E56FE46BE4C0E7F0E5C0E8F0C5D8DFC034
:1025D000E7F0E0C0E8F0060E0001E96FEA6B04DE08
:1025E00049C0E8FFE7DD4AC0E8FFE4DD4BC0E8FF93
:1025F000E1DD4CC0E8FFDEDD4DC0E8FFDBDD4EC0B5
:10260000E8FFD8DD0001E151D8A401D001D002D00B
:10261000E66B03D0060E0001E66F080ECBDD00016D
:10262000E651C8DD0E0E0001E227000EE323000E86
:10263000E35D3C0ED8B4E25DD8B001D001D003D048
:10264000400EE26FE36BE2C0E4F0E3C0E5F00001AE
:10265000E451ED6F050E5ED80001E551ED6F060EF9
:1026600059D81200FFFF9CD7FFFF36D0B6C5E8FF50
:10267000020D200EF324E96E010EF420EA6EEF50F5
:102680000001ED6F040E46D8240E0001ED6F000E20
:1026900041D80001C66B000EC66501D001D001D043
:1026A00019D00001C651020D210EF324E96E010E6E
:1026B000F420EA6EEF50D8B401D001D003D0C6C0E8
:1026C000B6F508D0010E0001C627000EC66501D080
:1026D00001D0E7D71200FFFFC9D7FFFF19D09568D7
:1026E000816AE00E936EF19E848284808484966A6F
:1026F00004D0D00E00018F6F03D0010E00018F6F48
:1027000001D000D000018F2FFCD784941200FFFF6E
:10271000E6D7ED00FFFF0DD0816E0001EE6FE00EF9
:10272000936EED51836E956A84928482956812004F
:10273000FFFFF2D7FFFF0ED09568816E0001EF6FAB
:10274000E00E936E84908350EE6F8480EE5100D043
:102750001200FFFFF1D7E700FFFF15D0E7C0E9F057
:10276000E8C0EAF0400E0001ED6F070ED3DF000174
:10277000E951ED6F080ECEDF0001EA51ED6F090E51
:10278000C9DF1200FFFFEAD7FFFF16D00001AE6FCE
:10279000AD6BAF6F00D00001AD51006EAE51016E58
:1027A000010EAD5F000EAE5B01500010D8A401D049
:1027B00001D0F1D71200FFFFE9D7A900FFFF10D029
:1027C000B5C5ACF0120E0001AB6FA951AB27AA51F1
:1027D000AC23ABC0E7F0ACC0E8F0BEDF1200FFFFF7
:1027E000EFD7B000FFFF1CD0E8CFB6F50001B46F03
:1027F000B6C5E8FF020D200EF324E96E010EF420A9
:10280000EA6EEF50B36F0E0EB26FB051B227B151F6
:10281000B323B2C0E7F0B3C0E8F09EDF1200FFFFC1
:10282000E3D7FFFF0DD0090E85DF8F6F080E82DF23
:102830008E6F8EC000F08FC001F000D01200FFFF3D
:10284000F2D78F00FFFF26D08FC0E9FF90C0EAFFCC
:10285000EECF1DF0EECF1EF0EECF1FF0EDCF20F04B
:10286000ED52ED5200011D0E916F000E926F17ECAC
:1028700027F00501DD6B64EC28F000C013F001C007
:1028800014F002C015F003C016F0010EE8CFDBF51E
:102890001200FFFFD9D7FFFF70D036D000011D0E08
:1028A0008F6F000E906F170E916F000E926F32ECCB
:1028B00027F0006E00C002F0036A03500210D8B483
:1028C00001D001D014D00001480E9F6FFF0EA06F01
:1028D000170EA16F000EA26F450EA36FA46B46ECFE
:1028E00018F0E8CFDCF5010EE8CFDDF501D011D00E
:1028F000DCC5DEF5CEEC10F00009D8B401D001D073
:1029000002D0000E38D005D0DDC5E8FF010AF0E0A6
:10291000C5D764EC28F013C0E8FF005C046E14C057
:10292000E8FF0158056E15C0E8FF0258066E16C094
:10293000E8FF0358076E000E075C08E1000E065C16
:1029400005E1010E055C02E12C0E045CD8A001D06B
:1029500001D00FD064EC28F000C013F001C014F0D7
:1029600002C015F003C016F0010EE8CFDBF5050E2E
:1029700002D0010E00D01200FFFF8FD79300FFFF9F
:102980003BD0DCC5E8FF160D6C0EF324E96E000E9B
:10299000F420EA6E450EEE6E000EED6E93C096F0DA
:1029A00094C097F000019551F6DA0501DA6B64ECFA
:1029B00028F000C013F001C014F002C015F003C0ED
:1029C00016F000019505D8A401D001D00BD0050167
:1029D000DA890001010E176F000E186F020EE8CFA2
:1029E000DDF508D00501DA990001176B186B030EAD
:1029F000E8CFDDF51200FFFFC4D7FFFF0DD0DAC529
:102A000000F000A801D001D003D007D803D002D035
:102A1000B3D900D01200FFFFF2D7FFFF36D100017B
:102A2000976B64EC28F013C0E8FF005C046E14C0E0
:102A3000E8FF0158056E15C0E8FF0258066E16C083
:102A4000E8FF0358076E000E075C08E1000E065C05
:102A500005E1010E055C02E12C0E045CD8A001D05A
:102A600001D00DD0010E0001976F64EC28F000C07A
:102A700013F001C014F002C015F003C016F0F3D03B
:102A800000019705D8A401D001D024D0976B05018F
:102A9000DB2BDB05006E030E005CD8A001D001D05B
:102AA00005D0010EE8CFDBF5050EEDD00001175182
:102AB000010A1811D8A401D001D003D0040EE3D02C
:102AC00009D00001010E175F000E185B050EE8CF5C
:102AD000DDF5D7D0DCC5E8FFCBEC19F00009D8A4B0
:102AE00001D001D001D0CDD00001940EA76F000E0F
:102AF000A86FE4EC19F00001930EA76F000EA86F09
:102B0000E4EC19F00001960EA76F000EA86FE4EC3C
:102B100019F00001950EA76F000EA86FE4EC19F0F4
:102B200000019351030A9411D8A401D001D02DD0F3
:102B300017C000F018C001F09651011802E195513C
:102B40000018D8A401D001D00BD00501DA93010EF2
:102B5000E8CFDBF5010EE8CFDDF5000E94D015D0FF
:102B600017C000F018C001F000010150965D02E1AD
:102B70000050955DD8B001D001D007D095C019F0B4
:102B800096C01AF0040EE8CFDDF540EC1AF0000113
:102B90009351050A9411D8A401D001D006D095C054
:102BA00011F096C012F0030E6ED06BD0DCC5DEF5CE
:102BB000CEEC10F00009D8B401D001D008D019C073
:102BC00098F01AC099F021DA020EE8CFDDF559D05D
:102BD000DCC5E8FFCBEC19F00009D8B401D001D076
:102BE0000DD064EC28F000C013F001C014F002C056
:102BF00015F003C016F0000E46D012D000011B5194
:102C00001C11D8A401D004D0020E1C6102D000D047
:102C100002D000D004D0060EE8CFDDF501D031D0CF
:102C2000DCC5DEF5CEEC10F00009D8B401D001D03F
:102C300018D017C098F018C099F0E7D90001010E1C
:102C40001727000E18230501DA83DDC5E8FF060A01
:102C5000D8A401D001D002D0020E15D0020EE8CFC8
:102C6000DDF50FD00ED0DDC5E8FF010AB1E0030AA3
:102C700001E106D7060A9AE0010AD2E0030AD0E091
:102C800000D0010E00D01200FFFFC9D6FFFF22D0F6
:102C90000001920EA76F000EA86FE4EC19F000017E
:102CA000010E1B27000E1C231CC0E8FF020AD8A43B
:102CB00001D001D00AD040EC1AF00501DA81000100
:102CC0001B6B1C6B050EE8CFDDF50001925100D0A7
:102CD0001200FFFFDDD7FFFF3ED0DAC500F000A8ED
:102CE00001D001D01CD0DAC500F000B001D001D075
:102CF00004D00501DA8140EC1AF0DAC500F000A238
:102D000001D001D006D00501DA850501DA9721D07E
:102D100005D0060EE8CFDDF50501DA871AD0DAC551
:102D200000F000B001D001D004D00501DA8146ECFA
:102D300019F0DAC500F000A201D001D005D00501DC
:102D4000DA850501DA9705D0030EE8CFDDF5050138
:102D5000DA871200FFFFC1D7FFFF0DD0DAC500F000
:102D600000A801D001D003D058DE03D002D004D88F
:102D700000D01200FFFFF2D7FFFFEBD00001976BEE
:102D800064EC28F013C0E8FF005C046E14C0E8FF98
:102D90000158056E15C0E8FF0258066E16C0E8FF20
:102DA0000358076E000E075C08E1000E065C05E1A3
:102DB000010E055C02E12C0E045CD8A001D001D00C
:102DC0000DD0010E0001976F64EC28F000C013F0E5
:102DD00001C014F002C015F003C016F0ACD0000121
:102DE0009751D8B401D001D012D00501DB2BDB05FF
:102DF000006E030E005CD8A001D001D006D0010EF9
:102E0000E8CFDBF5050EA3D002D0040EA0D0DCC5C0
:102E1000E8FFCBEC19F00009D8A401D001D001D013
:102E200094D00001940EA76F000EA86FE4EC19F087
:102E30000001930EA76F000EA86FE4EC19F00001DB
:102E4000960EA76F000EA86FE4EC19F00001950E26
:102E5000A76F000EA86FE4EC19F040EC1AF0000127
:102E60009351040A9411D8A401D001D022D017C0E4
:102E700000F018C001F09651011802E195510018B8
:102E8000D8A401D001D012D00501DA83010EE8CF19
:102E9000DBF5DAC500F000A601D001D004D00501B1
:102EA000DA85000E54D00501DD6B02D0010E4FD043
:102EB00010D000019351050A9411D8A401D001D07B
:102EC00007D095C011F096C012F0030E40D001D08B
:102ED0003CD0DCC5DEF5CEEC10F00009D8B401D052
:102EE00001D01CD00001010E1727000E1823000E80
:102EF000C5EC18F0030EC5EC18F018C0E8FFC5ECDF
:102F000018F017C0E8FFC5EC18F00501DA910501CB
:102F1000DA93010EE8CFDDF5000E19D016D0DCC52E
:102F2000DEF5CEEC10F00009D8B401D001D002D00B
:102F3000000E0DD00AD0DDC5E8FF000ACAE0010A84
:102F4000EEE0020A01E14BD700D0010E00D01200E2
:102F5000FFFF14D7FFFF1DD00001936F9351C5EC05
:102F600018F00001010E1B27000E1C231CC0E8FFF7
:102F7000020AD8A401D001D00AD046EC19F005010C
:102F8000DA8100011B6B1C6B030EE8CFDDF512002C
:102F9000FFFFE2D79600FFFF36D00001996F000EC9
:102FA000C5EC18F000019951C5EC18F096C0E9FF86
:102FB00097C0EAFFEF500001986F010E9627000EB0
:102FC00097239851C5EC18F000019851D8A401D06E
:102FD00001D0ECD76F0EC5EC18F0630EC5EC18F0FD
:102FE000740EC5EC18F0650EC5EC18F0740EC5EC47
:102FF00018F0000EC5EC18F046EC19F000011B6B40
:103000001C6B1200FFFFC9D79800FFFF12D0000E03
:10301000C5EC18F0040EC5EC18F000019951C5EC90
:1030200018F000019851C5EC18F046EC19F01200A8
:10303000FFFFEDD7FFFF28D000018E6B010E8E65DC
:1030400001D001D001D01ED000018E51160D6E0EA0
:10305000F324E96E000EF420EA6E000EEE6E000E10
:10306000ED6E8E51160D770EF324E96E000EF420EE
:10307000EA6EFE0EEF16010E8E27010E8E6501D050
:1030800001D0E2D71200FFFFD7D79F00FFFF69D022
:103090000001620EA66F000EA76FA56B010EA5655D
:1030A00001D001D001D059D0000100EE0CF0A651A2
:1030B000E926A751EA22EE50ED10D8A401D001D0A4
:1030C00040D000EE0CF0A651E926A751EA229FC09D
:1030D000EEFFA0C0EDFFA251A111D8B401D001D0E4
:1030E0000DD0A6C0C6F0A7C0C7F0A1C0C8F0A2C04E
:1030F000C9F00A0ECA6FCB6BC8EC02F0000100EEFB
:103100000AF0A651E926A751EA22A3C0EEFFA4C007
:10311000EDFF00EE0EF0A651E926A751EA22000EBF
:10312000EE6E000EED6E00EE10F0A651E926A751EE
:10313000EA22000EEE6E000EED6EA5C0DEF5A55182
:103140000ED0160E0001A627000EA723010EA527FC
:10315000010EA56501D001D0A7D7FF0E00D0120047
:10316000FFFF96D7FFFF10D000019F6F9F51160DF4
:103170006E0EF324E96E000EF420EA6EFF0EEE6E82
:10318000000EED6E1200FFFFEFD7FFFF7ED00001B3
:10319000A56FDEC5E8FF160D620EF324A16F000EC9
:1031A000F420A26F00EE0EF0A151E926A251EA220E
:1031B000EE50ED10D8A401D001D01FD000EE12F0D7
:1031C000A151E926A251EA22B6C5EFFF1C0EB06F4D
:1031D000B16B00EE12F0A151E926A251EA22EF50A4
:1031E000F2EC13F0000100EE13F0A151E926A25118
:1031F000EA22000EEE6E000EED6E0001A551DAEC33
:1032000010F0000100EE0EF0A151E926A251EA22D1
:10321000EECF00F0EDCF01F000EE13F0A151E92662
:10322000A251EA22EFCF02F0010EEE26EFCF03F01B
:10323000000EED220150035C02E10050025CD8A0B8
:1032400001D001D009D000EE0EF0A151E926A25123
:10325000EA22EE2A000EED22000100EE0EF0A1514E
:10326000E926A251EA22EECFA3F0EDCFA4F0030E9F
:10327000A45DD60ED8B4A35DD8A001D001D001D0F2
:1032800005D8010E00D01200FFFF81D7FFFF82D0CA
:10329000DEC5E8FF160D620EF3240001AE6F000ECE
:1032A000F420AF6F00EE0CF0AE51E926AF51EA22E8
:1032B000EECFE1F0EDCFE2F088EC1EF000C0A6F01A
:1032C00001C0A7F0000100EE0AF0AE51E926AF51AF
:1032D000EA22EECFE1F0EDCFE2F088EC1EF000C084
:1032E000A8F001C0A9F0000100EE0EF0AE51E926F1
:1032F000AF51EA22EECF00F0EDCF01F0080E00242E
:10330000AA6F000E0120AB6FAC6BAD6B140EB06FEB
:10331000B16B00EE12F0AE51E926AF51EA22EF5048
:10332000F2EC13F0AEC0C6F0AFC0C7F0110E000152
:10333000C86FAAC0C9F0ABC0CAF081EC22F0AAC025
:10334000E1F0ABC0E2F088EC1EF000C0AAF001C0D2
:10335000ABF00001A60EE76F000EE86F080EE96FF4
:10336000EA6BF4EC10F034EC13F0000100EE12F014
:10337000AE51E926AF51EA22FF0EEF6E00EE0EF0DD
:10338000AE51E926AF51EA22000EEE6E000EED6E50
:103390001200FFFF7DD7FFFF15D0E8CFDEF500015B
:1033A0009F6FDEC5E8FF160D720EF324E96E000E66
:1033B000F420EA6EEE50ED10000ED8A4010E00D0FD
:1033C0001200FFFFEAD7A700FFFF59D0DEC5E8FFD4
:1033D000160D720EF324E96E000EF420EA6EEE5024
:1033E000ED10D8A401D001D002D0000E46D0DEC529
:1033F000E8FF160D770EF324E96E000EF420EA6E56
:10340000EF50006E00A001D001D011D0DEC5E8FF62
:10341000160D770EF324E96E000EF420EA6EFE0E10
:10342000EF161C0E0001A96FAA6BDEEC13F050EC36
:1034300011F0A7C0E9FFA8C0EAFFEF6EDEC5E8FF04
:10344000160D720EF324E96E000EF420EA6EEE06FD
:10345000000EED5ADEC5E8FF160D720EF324E96E7C
:10346000000EF420EA6EEE50ED10D8A401D001D089
:1034700002D0C9EC11F0010E00D01200FFFFA6D758
:10348000FFFF20D0DEC5E8FF160D720EF324E96EB3
:10349000000EF420EA6EEE50ED10D8B401D001D049
:1034A00002D0C9EC11F0DEC5E8FF160D720EF32450
:1034B000E96E000EF420EA6E000EEE6E000EED6E68
:1034C0001200FFFFDFD79400FFFF66D00001980EC7
:1034D000CE6F000ECF6F080ED06FD16B67EC11F07E
:1034E00098C0E1F099C0E2F088EC1EF000C098F0BE
:1034F00001C099F09AC0E1F09BC0E2F088EC1EF0A8
:1035000000C09AF001C09BF09CC0E1F09DC0E2F0C9
:1035100088EC1EF0F80E002400019C6FFF0E0120C5
:103520009D6F9EC0E1F09FC0E2F088EC1EF000C0ED
:103530009EF001C09FF00001980EA16F000EA26FD7
:1035400094C0A3F095C0A4F029D80001A06FA029D1
:10355000D8A401D001D003D0C9EC11F019D00001DA
:10356000A051160D720EF324E96E000EF420EA6EDF
:103570009CC0EEFF9DC0EDFFA051160D770EF32409
:10358000E96E000EF420EA6EEF50FE0B0109EF6EBB
:10359000010E00D01200FFFF99D7A100FFFFBCD0A1
:1035A0000001A669620EA76F000EA86FA56B010E41
:1035B000A56501D001D001D080D0000110EE02F04D
:1035C000A151E126A251E22200EE0CF0A751E9261A
:1035D000A851EA22EE52E652E550ED18E7CFE8FF97
:1035E000D8B4EF18D8A401D001D05BD0A1C0E9FFB6
:1035F000A2C0EAFF10EE0AF0A751E126A851E2228C
:10360000E652EE52ED50E518EFCFE8FFD8B4E718D8
:10361000D8A40DD000D000EE10F0A751E926A85193
:10362000EA22EE50ED10D8A402D000D002D000D093
:1036300035D0000110EE06F0A351E126A451E2229C
:1036400000EE06F0A751E926A851EA22EE50E6184E
:1036500008E1EE50E61805E1EE50E61802E1EE5002
:10366000E618D8A401D014D000EE06F0A751E92640
:10367000A851EA22FF0EEE18FF0ED8B4EE18FF0E86
:10368000D8B4EE18FF0ED8B4EE18D8A402D000D0EB
:1036900002D000D003D00001A5513CD00001A551BB
:1036A000A66F160E0001A727000EA823010EA5275E
:1036B000010EA56501D001D080D70001A629D8B49C
:1036C00001D001D024D0A651160D620EF324A76FAD
:1036D000000EF420A86FA7C0C6F0A8C0C7F0A3C012
:1036E000C8F0A4C0C9F00A0ECA6FCB6BC8EC02F0D8
:1036F000A1C0E9FFA2C0EAFF000110EE0AF0A75145
:10370000E126A851E222EECFE6FFEDCFE5FF000172
:10371000A65100D01200FFFF43D7B900FFFF000100
:10372000C76BC86BB9C0C5F0BAC0C6F00001BDC058
:10373000F6FFBEC0F7FFBD2B000EBE23050EF764DB
:1037400004D00800FFFFF55005D0F6CFE9FFF7CF12
:10375000EAFFEF50C26FC2510001D8B4C7D2250AA8
:10376000D8B40BD0C72B000EC823BC51BB11D8A4B2
:103770007BD1C251BEEC28F0D9D70001C069C16B22
:10378000BF6B62D20001BC51BB11D8A4B3D2B8D276
:10379000C5C0E9FFC6C0EAFF0001020EC527000E42
:1037A000C623EF5095D20001BF8D4ED20001BF2B32
:1037B00006D0080E0001C027FE0E0001C027C5C0BC
:1037C000E9FFC6C0EAFF0001020EC527000EC623AE
:1037D000EECFC3F0EDCFC4F0BFA10DD0C4AF06D083
:1037E000C36DC41FD8B0C42BC10707D00001BF915F
:1037F000BFAD03D0F9D70001BF910B0E0001C02768
:10380000C0C002F0036AC3C000F0C4C001F022ECE3
:1038100028F000500001C26FC0C002F0036AC3C0AC
:1038200000F0C4C001F022EC28F004C0C3F005C0D1
:10383000C4F0010EC96FCA6B0001CA51C45D02E138
:10384000C951C35DD8A010D0C0C002F0036AC9C07E
:1038500000F0CAC001F095EC28F004C0C9F005C022
:10386000CAF00001C107E8D70001BFA916D01CD0DB
:103870000001C72B000EC823BC51BB11D8B40AD01D
:10388000BBC0E9FFBCC0EAFF200EEF6EBB2B000EF1
:10389000BC2303D0200EBEEC28F00001C107C151AB
:1038A000800A7F0FD8B0E4D70001BFA115D0C72B85
:1038B000000EC823BC51BB11D8B40AD0BBC0E9FF6D
:1038C000BCC0EAFF2D0EEF6EBB2B000EBC2317D041
:1038D0002D0EBEEC28F013D00001BFAD10D0C72BC9
:1038E000000EC823BC51BB11D8B406D0BBC0E9FF41
:1038F000BCC0EAFF2B0EE7D72B0EBEEC28F0000170
:10390000BFB916D051D00001C72B000EC823BC513F
:10391000BB11D8B40AD0BBC0E9FFBCC0EAFF300E6F
:10392000EF6EBB2B000EBC2303D0300EBEEC28F094
:103930000001C107C151800A7F0FD8A035D0E3D75D
:10394000C9C002F0CAC003F0C3C000F0C4C001F097
:1039500022EC28F004C000F005C001F0C0C002F065
:10396000036A22EC28F000500001C16F800A760F34
:10397000D8A002D0070EC1270001C72B000EC82314
:10398000BC51BB11D8B40BD0C151300FBBC0E9FF43
:10399000BCC0EAFFEF6EBB2B000EBC2305D00001BC
:1039A000C151300FBEEC28F0C0C002F0036AC90E4E
:1039B000E96E000EEA6EEE50006EEF50016E22ECE2
:1039C00028F00550ED6E0450EF6EEE50ED10D8A4C7
:1039D000B7D7090E0001C26502D0070EC227000149
:1039E000C72B000EC823BC51BB11D8B408D0C2519C
:1039F000300FBBC0E9FFBCC0EAFFEF6E3BD0000157
:103A0000C251300FBEEC28F091D60001C151800A9E
:103A10007E0FD8A017D0C72B000EC823BC51BB11F6
:103A2000D8B40AD0BBC0E9FFBCC0EAFF200EEF6EDD
:103A3000BB2B000EBC2303D0200EBEEC28F00001EF
:103A4000C107E3D7C5C0E9FFC6C0EAFF0001020E07
:103A5000C527000EC623EF50C26FC72B000EC82328
:103A6000BC51BB11D8B40AD0BBC0E9FFBCC0EAFF4F
:103A7000C2C0EFFFBB2B000EBC2358D60001C251C1
:103A8000BEEC28F053D6C5C0E9FFC6C0EAFF00016E
:103A9000020EC527000EC623EECF00F0EDCF01F0D9
:103AA00000C01EF101C01FF1D96A1EC100F01FC184
:103AB00001F0D9500024026E000E0120036E02C0F6
:103AC000F6FF03C0F7FF050EF76404D00800FFFF00
:103AD000F55005D0F6CFE9FFF7CFEAFFEF50000928
:103AE000D8B402D0D92AE1D70001C051D96002D0A0
:103AF000D950C06F0001C051C1BF46D0FF0AC125D7
:103B0000D8A042D0C72B000EC823BC51BB11D8B4DB
:103B10000AD0BBC0E9FFBCC0EAFF200EEF6EBB2B92
:103B2000000EBC2303D0200EBEEC28F00001C1071C
:103B3000E1D71EC1F6FF1FC1F7FF050EF76404D0E1
:103B40000800FFFFF55005D0F6CFE9FFF7CFEAFFF9
:103B5000EF500001C26F01011E2B000E1F23000158
:103B6000C72BC823BC51BB11D8B40AD0BBC0E9FFD6
:103B7000BCC0EAFFC2C0EFFFBB2B000EBC2304D0C9
:103B80000001C251BEEC28F00001C007C029D8B422
:103B9000CDD5CFD7BDC0F6FFBEC0F7FF050EF76489
:103BA00004D00800FFFFF55005D0F6CFE9FFF7CFAE
:103BB000EAFFEF502A0AD8A40FD0C5C0E9FFC6C05B
:103BC000EAFF0001020EC527000EC623EF50C06FAA
:103BD000BD2B000EBE2338D0BDC0F6FFBEC0F7FF20
:103BE000050EF76404D00800FFFFF55005D0F6CFAE
:103BF000E9FFF7CFEAFFEF50D00F0001C06FBD2BF8
:103C0000000EBE23BDC0F6FFBEC0F7FF050EF76471
:103C100004D00800FFFFF55005D0F6CFE9FFF7CF3D
:103C2000EAFFEF50D96E2F0ED9640ED03A0ED9604C
:103C30000BD00001C0510A0DD950F324D00FC7D7C3
:103C40000001BFB538D0BF890001BDC0F6FFBEC0BE
:103C5000F7FFBD2B000EBE23050EF76404D008004D
:103C6000FFFFF55005D0F6CFE9FFF7CFEAFFEF50A1
:103C7000C26F000A01E186D52A0A01E189D5010A4D
:103C800001E191D5050A86E01E0ADAE0680A01E141
:103C900090D53B0A01E1B9D6070A01E187D50B0AA5
:103CA00001E18AD51C0A01E1EED6060A01E187D5B9
:103CB0000D0A01E17ED52F0E0001C2650BD03A0E30
:103CC000C26108D0BF85C1510A0DC251F324D00F83
:103CD000C16FBAD70001C72B000EC823BC51BB115E
:103CE000D8A4C2D6C251BEEC28F020D5BC51BB111D
:103CF000D8B406D0BBC0E9FFBCC0EAFF000EEF6A33
:103D0000C7C000F0C8C001F01200FFFF08D5E100F5
:103D1000FFFF12D0E1C0E3F0E2C0E4F00001E451A3
:103D2000E56FE351E46FE551E36FE3C000F0E4C0F9
:103D300001F000D01200FFFFEDD78E00FFFF50D042
:103D40008EC08FF08FC090F090C091F091C092F033
:103D500000018F0E936F000E946F00EE03F09351ED
:103D6000E9269451EA22EF508E6F93C0E9FF94C088
:103D7000EAFF10EE03F09351E1269451E222EFCFD7
:103D8000E7FF93C0E9FF94C0EAFF8EC0EFFF00EEAB
:103D900002F09351E9269451EA22EF508E6F10EE13
:103DA00001F09351E1269451E22200EE02F093518A
:103DB000E9269451EA22E7CFEFFF00EE01F093519C
:103DC000E9269451EA228EC0EFFF8FC000F090C028
:103DD00001F091C002F092C003F000D01200FFFF8A
:103DE000AFD7DF00FFFF78D00001EB6BEC6BED6B22
:103DF000EE6BD890E231E46FE131E36FDFC0E5F0C4
:103E0000E0C0E6F017D0E5C0E9FFE6C0EAFF000138
:103E1000020EE527000EE623EECF00F0EDCF01F015
:103E2000026A036A0050EB270150EC230250ED2395
:103E30000350EE230001E351006EE451016E010EC8
:103E4000E35F000EE45B01500010D8A401D001D064
:103E5000DAD70001E1A101D001D00DD0E5C0E9FF22
:103E6000E6C0EAFFEF50EB27010ED8B0EC27D8B040
:103E7000ED27D8B0EE27EBC0E7F0ECC0E8F0EDC0DE
:103E8000E9F0EEC0EAF015D00001ED6BEE6BEB51FE
:103E9000E325EB6FEC51E421EC6FED6BD8B0ED2B2B
:103EA000EE6BEBC0E7F0ECC0E8F0EDC0E9F0EEC07F
:103EB000EAF0E9C0E3F0EAC0E4F00001E451E31104
:103EC000D8A401D001D0E0D70001EB1D006EEC1D9D
:103ED000016E00D01200FFFF87D78E00FFFF2FD0AA
:103EE0008EC08FF08FC090F017D0600E00018E65ED
:103EF00006D000D07B0E8E6102D000D002D000D060
:103F000006D08FC0E9FF90C0EAFFE00EEF26010E59
:103F100000018F27000E90238FC0E9FF90C0EAFFB9
:103F2000EF5000018E6F8E51D8A401D001D0DDD7A3
:103F30008EC000F08FC001F000D01200FFFFD0D77C
:103F40008E00FFFF34D090C090F091C091F08EC0F1
:103F50008EF08FC08FF01DD090C0F6FF91C0F7FF9C
:103F60008EC0E9FF8FC0EAFF050EF76403D008009A
:103F7000F55005D0F6CFE1FFF7CFE2FFE750EF6E47
:103F8000010E00018E27000E8F23010E9027000ED8
:103F90009123000192079229D8A401D001D0DCD747
:103FA0008EC000F08FC001F000D01200FFFFCBD711
:103FB000FFFF23D00001906F17D0040E00018F6F18
:103FC0000CD0500E0001916F03D0010E0001916FD3
:103FD00001D000D00001912FFCD700018F078F295D
:103FE000D8A401D001D0EDD7000190079029D8A422
:0C3FF00001D001D0E2D71200FFFFDCD7A7
:104000009F00FFFF94D00001A30ECE6F000ECF6F74
:104010001C0ED06FD16B67EC11F0C9EC11F00001F0
:10402000A30EBF6F000EC06F4CD900EEA3F0EE5090
:10403000010AED10D8B401D006D00001A751060A3C
:10404000D8B402D000D007D000D00001A851040A93
:10405000D8B402D000D002D000D002D0000E65D07B
:1040600000EEA9F0EE50020AED10D8A401D001D064
:1040700007D0A1C0E9FFA2C0EAFF000EEF6E18D082
:1040800000EEA9F0EE50010AED10D8A401D001D045
:1040900007D0A1C0E9FFA2C0EAFF010EEF6E08D071
:1040A000A1C0E9FFA2C0EAFF020EEF6E000E3DD0F4
:1040B00045C0E8FF0001BB6307D000D046C0E8FF61
:1040C000BC6302D000D001D007D047C0E8FF000198
:1040D000BD6302D000D001D007D048C0E8FF000186
:1040E000BE6302D000D002D000D01DD0AB0EE96E6E
:1040F000000EEA6E9FC0E1FFA0C0E2FF060EB8EC22
:1041000028F0000100EE06F09F51E926A051EA22B6
:10411000B1C0EEFFB2C0EEFFB3C0EEFFB4C0EEFF21
:10412000010E03D002D0000E00D01200FFFF6BD7AB
:104130009F00FFFFC4D0010E0001A26FA36B000E11
:10414000A46F080EA56F060EA66F040EA76FA1053B
:10415000D8A401D001D00AD0010EA86FA96BB46910
:10416000B569B669B769B869B9690FD0020E0001BF
:10417000A86FA96B9FC0E9FFA0C0EAFFB40EE16E73
:10418000000EE26E060EB8EC28F049C0AAF04AC054
:10419000ABF04BC0ACF04CC0ADF04DC0AEF04EC07B
:1041A000AFF045C0B0F046C0B1F047C0B2F048C073
:1041B000B3F04FC000F0000100EE06F09F51E92679
:1041C000A051EA22EF50B019016E0050011400090D
:1041D000D8B401D011D050C000F000EE07F09F51CC
:1041E000E926A051EA22EF50B119016E00500114E6
:1041F0000009D8B402D000D013D000D051C000F0D4
:10420000000100EE08F09F51E926A051EA22EF508C
:10421000B219016E005001140009D8B402D000D0C8
:1042200013D000D052C000F0000100EE09F09F5101
:10423000E926A051EA22EF50B319016E0050011493
:104240000009D8B402D000D002D000D009D053C0A9
:10425000BAF054C0BBF055C0BCF056C0BDF00FD092
:10426000000100EE06F09F51E926A051EA22EECFB0
:10427000BAF0EECFBBF0EECFBCF0EECFBDF0000158
:10428000A20EBF6F000EC06F1CD80001B40EDF6F0E
:10429000000EE06F060EE16F1C0EE26FE36BCEECDA
:1042A00012F00001A20EE76F000EE86F1C0EE96F1E
:1042B000EA6BF4EC10F034EC13F01200FFFF3BD784
:1042C000BF00FFFF43D0BFC0E9FFC0C0EAFFEECF91
:1042D000E1F0EDCFE2F088EC1EF0BFC0E9FFC0C016
:1042E000EAFF00C0EEFF01C0EDFF000100EE02F0AA
:1042F000BF51E926C051EA22EECFE1F0EDCFE2F066
:1043000088EC1EF0000100EE02F0BF51E926C0511A
:10431000EA2200C0EEFF01C0EDFF00EE06F0BF5143
:10432000E926C051EA22EECFE1F0EDCFE2F088ECD1
:104330001EF0000100EE06F0BF51E926C051EA224E
:1043400000C0EEFF01C0EDFF1200FFFFBCD79400DC
:10435000FFFFD5D00001A40ECE6F000ECF6F140E5C
:10436000D06FD16B67EC11F00001A451F00B400A43
:10437000D8B401D001D001D0BCD0A4C000F00F0E41
:104380000016D8900036D8900034EC0F0001B86FBA
:10439000140EB86501D001D001D0ABD00001B851E6
:1043A000D8B401D001D009D0B90ECE6F000ECF6FB6
:1043B000B851D06FD16B67EC11F0AEC09CF0AFC0BC
:1043C0009DF00001AE6BAF6BA40EDF6F000EE06FCF
:1043D000140EE16FE26BF2EC1EF0001C026E011C89
:1043E000036E02C0A0F003C0A1F00001B851D8B420
:1043F00001D001D012D0B90EDF6F000EE06FB851BE
:10440000E16FE26BF2EC1EF0001C026E011C036E09
:1044100002C0A2F003C0A3F003D00001A26BA36B03
:104420000001A00EDF6F000EE06F040EE16FE26B83
:10443000F2EC1EF000C09EF001C09FF00001A40E3F
:10444000DF6F000EE06FC5D800019F519D1902E19A
:104450009E519C19D8B401D006D0A451F00B400A4B
:10446000D8B402D000D002D000D001D042D0000198
:1044700095519411D8B401D001D00CD094C0E9FF6B
:1044800095C0EAFFB4C0EEFFB5C0EEFFB6C0EEFFC8
:10449000B7C0EEFF000100EE06F09651E9269751F5
:1044A000EA22B0C0EEFFB1C0EEFFB2C0EEFFB3C073
:1044B000EEFF98C0E9FF99C0EAFFADC0EFFFB85129
:1044C00000EEA6F0EECF00F0EDCF01F0005E000EA2
:1044D000015AEC0E0024006EFF0E0120016E9AC0FE
:1044E000E9FF9BC0EAFF00C0EEFF01C0EDFF010E37
:1044F00004D0C9EC11F0000E00D01200FFFF2AD743
:10450000C600FFFF64D0450E0001CB6FCC6B140ECC
:10451000C925CD6F000ECA21CE6F0101010E2227E1
:10452000000E232300EECFF022C1EEFF23C1EDFFEA
:104530000001D16BD26B640ED36FC851D46FD56BB1
:10454000D66B45C0D7F046C0D8F047C0D9F048C0B8
:10455000DAF000EE06F0C651E926C751EA22EECFA6
:10456000DBF0EECFDCF0EECFDDF0EECFDEF0CB0E09
:10457000DF6F000EE06F2DD80001CB0EDF6F000E55
:10458000E06F140EE16FE26BF2EC1EF000C0D5F0AC
:1045900001C0D6F0C6C0DFF0C7C0E0F00001E16B9B
:1045A000140EC925E26F000ECA21E36FCEEC12F0A3
:1045B0000001CB0EE76F000EE86F140EE96FEA6B97
:1045C000F4EC10F0006A016A00D01200FFFF9BD7E4
:1045D000DF00FFFF48D0000100EE02F0DF51E926C6
:1045E000E051EA22EECFE1F0EDCFE2F088EC1EF0F0
:1045F000000100EE02F0DF51E926E051EA2200C09E
:10460000EEFF01C0EDFF00EE04F0DF51E926E051BE
:10461000EA22EECFE1F0EDCFE2F088EC1EF00001EF
:1046200000EE04F0DF51E926E051EA2200C0EEFF7F
:1046300001C0EDFF00EE0AF0DF51E926E051EA2269
:10464000EECFE1F0EDCFE2F088EC1EF0000100EEDD
:104650000AF0DF51E926E051EA2200C0EEFF01C076
:10466000EDFF1200FFFFB7D7FFFF0CD00501B86BBD
:104670000501B98102EC10F0A0EC26F01AEC18F05C
:104680001200FFFFF3D7FFFF2ED1010E0001936F41
:1046900018D10001936BFFD00001060E946F010E3C
:1046A000956F920E966F000E976F17EC12F0006EDA
:1046B00000C002F0036A03500210D8A401D001D058
:1046C00001D0FFD0010E0001936F9251D8A401D008
:1046D00001D004D0020EE8CFB8F50DD00001925100
:1046E000060AD8A401D001D004D0050EE8CFB8F551
:1046F00002D0C9EC11F0E5D00001936BBEEC26F0BE
:104700000009D8B401D001D002D00501B86BD9D0CE
:1047100000018E0E946F000E956F060E966F010EBF
:10472000976F920E986F000E996F000E9A6F010EA0
:104730009B6FA8EC21F0006E00C002F0036A0350EA
:104740000210D8B401D001D01ED0010E0001936F29
:104750009205D8A401D001D004D0030EE8CFB8F55B
:1047600011D000019251110AD8A401D001D004D077
:10477000070EE8CFB8F506D00001936BC9EC11F035
:104780000501B86B04D0C9EC11F00501B86B99D0E4
:104790000001060E946F010E956F00EE96F000C1B9
:1047A000EEFF01C1EDFF64EC1AF0006E00C002F0F4
:1047B000036A03500210D8B401D001D002D0050121
:1047C000B86B0001936B7DD00501B86B0101000E41
:1047D000015D2A0ED8B4005DD8B001D001D033D02D
:1047E0000001920E946F000E956FBA0E966F050E33
:1047F000976F000E986F010E996F020E9A6F010E5F
:104800009B6F040E9C6F010E9D6F75EC24F0006E83
:1048100000C002F0036A03500210D8B401D001D0E6
:1048200010D000019251080AD8A401D001D006D0BE
:10483000010E936F040EE8CFB8F502D00501B86BF6
:1048400002D00501B86BC9EC11F03BD0CEEC10F0F2
:104850000009D8B401D001D01CD00001060E946F1D
:10486000010E956F966BBA0E976F050E986F00C18B
:1048700099F000EE9AF002C1EEFF03C1EDFF00EEE9
:104880009CF004C1EEFF05C1EDFFFBEC24F0050137
:10489000B86B17D016D0B8C5E8FF000A01E1FCD606
:1048A000010A01E1F9D6030A01E132D7010A8CE0DD
:1048B000070ACCE0010A01E11FD7020A01E168D72B
:1048C00000D000019351D8A401D001D0E2D6BFECB2
:1048D0000BF094C500F000A001D001D002D005017A
:1048E000B9911200FFFFD1D69400FFFF82D00001E2
:1048F0009E0ECE6F000ECF6F080ED06FD16B67EC9F
:1049000011F0A0C0CCF0A1C0CDF00001A06BA16B54
:104910009E0EDF6F000EE06F080EE16FE26BF2ECAF
:104920001EF0001C026E011C036E02C0C6F003C024
:10493000C7F098C0E9FF99C0EAFFF80EEF2696C0CD
:10494000CEF097C0CFF098C0E9FF99C0EAFFEF50D2
:104950000001D06FD16B67EC11F096C0DFF097C00B
:10496000E0F098C0E9FF99C0EAFFEF500001E16F65
:10497000E26BF2EC1EF0001C026E011C036E02C022
:10498000C8F003C0C9F00001C60EDF6F000EE06F73
:10499000040EE16FE26BF2EC1EF000C0CAF001C041
:1049A000CBF000019E0ECE6F000ECF6F7AD894C070
:1049B000E9FF95C0EAFF9EC0EFFF9AC0E9FF9BC0E8
:1049C000EAFFA2C0EEFFA3C0EDFF9CC0E9FF9DC0BF
:1049D000EAFFA4C0EEFFA5C0EDFF0001CD51CB1949
:1049E00002E1CC51CA19000ED8B4010E00D0120059
:1049F000FFFF7DD79400FFFF52D000019F6B9651BF
:104A00009E6FA06BA16B9AC0A2F09BC0A3F09CC04C
:104A1000A4F09DC0A5F0A60EC66F000EC76F97C08C
:104A2000C8F098C0C9F09951CA6FCB6BC8EC02F0BE
:104A300000019E0ECE6F000ECF6F33D800019E0E88
:104A4000DF6F000EE06F080E9925E16FE26B000E3C
:104A5000E223F2EC1EF000C0A0F001C0A1F094C06F
:104A6000C6F095C0C7F0010E0001C86F080E992569
:104A7000C96FCA6B000ECA2381EC22F000019E0EA2
:104A8000E76F000EE86F080E9925E96FEA6B000EDC
:104A9000EA23F4EC10F034EC13F01200FFFFADD772
:104AA000CE00FFFF48D0000100EE04F0CE51E92611
:104AB000CF51EA22EECFE1F0EDCFE2F088EC1EF02C
:104AC000000100EE04F0CE51E926CF51EA2200C0E9
:104AD000EEFF01C0EDFF00EE06F0CE51E926CF510A
:104AE000EA22EECFE1F0EDCFE2F088EC1EF000011B
:104AF00000EE06F0CE51E926CF51EA2200C0EEFFCB
:104B000001C0EDFF00EE02F0CE51E926CF51EA22BE
:104B1000EECFE1F0EDCFE2F088EC1EF0000100EE08
:104B200002F0CE51E926CF51EA2200C0EEFF01C0CB
:104B3000EDFF1200FFFFB7D7FFFF3AD0F00E83164C
:104B40000F0E9512959A9598929A839A8398809AC7
:104B50009BEC0BF0F00E9516F00E83168382808A84
:104B6000ABEC0BF0809AA3EC0BF0F00E8316838273
:104B7000808AABEC0BF0809AABEC0BF0F00E831656
:104B80008382808AABEC0BF0809A0F0E9512280E70
:104B900010D8280E0ED8080E0CD80C0E0AD8010E0C
:104BA00008D8130E06D8800E04D800D01200FFFFDC
:104BB000C5D7FFFF2CD00001B96F00D029D800095C
:104BC000D8A401D001D0FAD7959A9598F00E9516F1
:104BD000F00E83160001B9390F0B8312839A839864
:104BE000ABEC0BF0808AABEC0BF0809AF00E8316E6
:104BF0000001B9510F0B8312ABEC0BF0808AABECC8
:104C00000BF0809A0F0E951200D01200FFFFD3D741
:104C1000FFFF24D0838A8398959A9598ABEC0BF08C
:104C2000808AABEC0BF083A601D001D00BD0809A28
:104C3000ABEC0BF0808AABEC0BF0809A839A010E00
:104C40000BD00AD0809AABEC0BF0808AABEC0BF067
:104C5000809A839A000E00D01200FFFFDBD7B900C4
:104C6000FFFF17D008D00001BB513AD8010E000158
:104C7000B927000EBA23B9C0E9FFBAC0EAFFEF5066
:104C80000001BB6FBB51D8A401D001D0ECD71200FA
:104C9000FFFFE8D7B900FFFF22D008D00001BB51C9
:104CA0001FD8010E0001B927000EBA23B9C0F6FFC4
:104CB000BAC0F7FF050EF76404D00800FFFFF550F7
:104CC00005D0F6CFE9FFF7CFEAFFEF500001BB6F49
:104CD000BB51D8A401D001D0E1D71200FFFFDDD72E
:104CE000FFFF2DD00001BC6F00D092DF0009D8A4D7
:104CF00001D001D0FAD7959A9598F00E9516F00E3E
:104D000083160001BC390F0B0F0B83128388839A23
:104D1000ABEC0BF0808AABEC0BF0809AF00E8316B4
:104D20000001BC510F0B8312ABEC0BF0808AABEC93
:104D30000BF0809A0F0E951200D01200FFFFD2D711
:104D4000FFFF1BD00501B26BFF0EE8CF10F1FF0E85
:104D5000E8CF11F1FF0EE8CF12F1FF0EE8CF13F10B
:104D6000FF0EE8CF14F1FF0EE8CF15F10101166B2D
:104D7000176B186B196B1200FFFFE4D7FFFF55D0BC
:104D80004BD00001940E9F6F000EA06F9E0EA16F7E
:104D9000000EA26F01EC20F0006E00C002F0036A6A
:104DA00003500210D8A401D001D001D03AD00001A4
:104DB0009E51D8A401D001D016D094C010F195C056
:104DC00011F196C012F197C013F198C014F199C077
:104DD00015F19AC016F19BC017F19CC018F19DC047
:104DE00019F11FD003D0010EE8CFB2F5CEEC10F0D0
:104DF0000009D8B401D001D00BD00001940E9F6FF0
:104E0000000EA06FA16B99EC20F00501B26B02D0EF
:104E1000000E09D006D005D0B2C5E8FF000AB1E007
:104E2000E5D7010E00D01200FFFFAAD79100FFFFC7
:104E300017D091C0E9FF92C0EAFFEECF99F0EECF14
:104E40009AF0EECF9BF0EECF9CF00001930E9F6F97
:104E5000000EA06F010EA16F99EC20F01200FFFF71
:104E6000E8D78F00FFFF43D08FC0E9FF90C0EAFF73
:104E700001011651EE1808E11751EE1805E118511D
:104E8000EE1802E11951EE18D8A401D01CD053C07D
:104E9000E8FF166307D000D054C0E8FF176302D0C4
:104EA00000D001D007D055C0E8FF0101186302D03F
:104EB00000D001D007D056C0E8FF0101196302D02D
:104EC00000D001D001D002D000D00DD0100EE96E7C
:104ED000010EEA6E91C0E1FF92C0E2FF060EB8EC4F
:104EE00028F0010E02D0000E00D01200FFFFBCD748
:104EF000B400FFFF04D00001B42B000EB523B4C0F2
:104F0000F6FFB5C0F7FF050EF76404D00800FFFFF9
:104F1000F55005D0F6CFE9FFF7CFEAFFEF50200AB2
:104F2000D8B4E9D7B4C0F6FFB5C0F7FF050EF764F3
:104F300004D00800FFFFF55005D0F6CFE9FFF7CF0A
:104F4000EAFFEF50090A0001D8B4D6D7B76BB86BA7
:104F5000B66BB4C0F6FFB5C0F7FF050EF76404D01A
:104F60000800FFFFF55005D0F6CFE9FFF7CFEAFFC5
:104F7000EF502D0AD8A403D0010EB62B15D0B4C023
:104F8000F6FFB5C0F7FF050EF76404D00800FFFF79
:104F9000F55005D0F6CFE9FFF7CFEAFFEF502B0A27
:104FA000D8A405D0010E0001B427000EB523B4C06B
:104FB000F6FFB5C0F7FF050EF76404D00800FFFF49
:104FC000F55005D0F6CFE9FFF7CFEAFFEF5085ECBB
:104FD00028F0D8A027D00A0E026E036AB7C000F0EE
:104FE000B8C001F095EC28F0B4C0F6FFB5C0F7FFEB
:104FF000050EF76404D00800FFFFF55005D0F6CF8A
:10500000E9FFF7CFEAFFEF500424006E000E052001
:10501000016ED00E00240001B76FFF0E0120B86FA3
:10502000010EC2D70001B651B7C000F0B8C001F000
:10503000D8B405D0001E011E002AD8B4012A1200DF
:10504000FFFF58D7FFFF066AFFFF046A056A025098
:10505000031003E1006A016A000C1F0E0612D890CB
:10506000062A02360336FCE3033202320250005CA9
:105070000350015804E3016E0250005ED8800436EC
:105080000536062E06BAF0D706AE05D0041E042A51
:10509000D8B40506051E0450026E0550036E06AC1A
:1050A000000C001E002AD8B40106011E000CFFFFF0
:1050B0000AD03C0ED66ED768070ED56ED58EF28418
:1050C000F28A1200FFFFF5D7FFFF0BD01AC100F0E4
:1050D0001BC101F01CC102F01DC103F000D0120081
:1050E000FFFFF4D7FFFF10D0F2A401D001D00AD007
:1050F000D7683C0ED66E01011A2B000E1B231C2311
:105100001D23F2941200FFFFEFD7FFFFD96E390E77
:10511000D96401D006D0300ED96001D002D0D88039
:1051200001D0D8901200FFFFF1D7FFFF025000021C
:10513000F3CF04F0F4CF05F00102F350052603503D
:105140000002F350052612000900F5CFEEFFFFFF25
:10515000EA50E262F9D7E950E162F6D71200EE6A4E
:10516000FFFFEA50E262FBD7E950E162F8D7120094
:10517000FFFFEECFE6FFE82EFBD7000CFFFF12008B
:04518000FFFFFDD759
:020000040030CA
:04000000FFFAFCFE09
:020000040000FA
:00000001FF
